:020000040800F2
:1000000000060020E1020008E3020008E302000805
:10001000E3020008E3020008E3020008E30200082C
:10002000E3020008E3020008E30200084933000885
:10003000E3020008E3020008E3020008E30200080C
:10004000E3020008E3020008E3020008E3020008FC
:10005000E3020008E3020008354B0008614B00088A
:100060008D4B0008B94B0008E54B0008D51100087E
:10007000FD1100082912000855120008811200081D
:10008000A9120008D5120008E3020008E3020008E4
:10009000E3020008E3020008E3020008114C000834
:1000A000E3020008E3020008E3020008E30200089C
:1000B000E3020008E3020008E3020008E30200088C
:1000C000E3020008E3020008E3020008E30200087C
:1000D000E3020008FD4C0008E3020008114D00088F
:1000E000754C0008E3020008E3020008E302000880
:1000F000E3020008E3020008E3020008011300081D
:10010000E3020008E30200084D4D0008E302000886
:10011000E3020008254D0008E3020008E30200089E
:100120002D1300085513000881130008AD130008B3
:10013000D9130008E3020008E3020008E302000804
:10014000E3020008E3020008E3020008E3020008FB
:10015000011400082D14000859140008E3020008D7
:10016000E3020008E3020008E3020008E3020008DB
:10017000E3020008353F0008E3020008E30200083C
:10018000E3020008E3020008394D0008E30200081A
:10019000E3020008E3020008E3020008E3020008AB
:1001A000E3020008E3020008E3020008E30200089B
:1001B000E3020008E3020008E3020008E30200088B
:1001C000E3020008E3020008E3020008E30200087B
:1001D000E3020008213F0008E3020008E3020008F0
:1001E000E3020008E3020008E3020008E30200085B
:1001F000E3020008E3020008E3020008E30200084B
:10020000E3020008E3020008E3020008E30200083A
:10021000E3020008E3020008E3020008E30200082A
:10022000E3020008E3020008E3020008E30200081A
:10023000E94C0008E3020008E3020008E3020008BA
:10024000E3020008E3020008E3020008E3020008FA
:10025000E3020008E3020008E3020008E3020008EA
:10026000E3020008E3020008E3020008E3020008DA
:10027000E3020008E3020008E3020008E3020008CA
:10028000E3020008E3020008E3020008E3020008BA
:10029000E3020008E3020008E3020008E3020008AA
:1002A000E3020008E3020008E3020008E30200089A
:1002B000E3020008E3020008E3020008E30200088A
:1002C000E3020008E3020008E3020008E30200087A
:1002D000E3020008E3020008E3020008E30200086A
:1002E00002E000F000F8FEE772B6374880F30888B5
:1002F000364880F3098836483649086040F20000E5
:10030000CCF200004EF63471CEF200010860BFF36B
:100310004F8FBFF36F8F40F20000C0F2F0004EF637
:100320008851CEF200010860BFF34F8FBFF36F8F8B
:100330004FF00000E1EE100A4EF63C71CEF20001E3
:100340000860062080F31488BFF36F8F03F05EF817
:1003500004F0A6F94FF055301F491B4A91423CBFAB
:1003600041F8040BFAE71D49184A91423CBF41F895
:10037000040BFAE71A491B4A1B4B9A423EBF51F83D
:10038000040B42F8040BF8E700201849184A914280
:100390003CBF41F8040BFAE703F076F804F004FAE6
:1003A000144C154DAC4203DA54F8041B8847F9E7A6
:1003B00000F042F8114C124DAC4203DA54F8041B21
:1003C0008847F9E703F05EB800060020002200200D
:1003D0000000000808ED00E00000002000060020FA
:1003E000385E0008002200206C22002070220020CD
:1003F000B4580020E0020008E0020008E002000813
:10040000E00200082DE9F04F2DED108AC1F80CD064
:10041000D0F80CD0BDEC108ABDE8F08F002383F338
:1004200011882846A047002002F0FCF9FEE702F000
:1004300087F900DFFEE7000038B500F0D3FC00F0DC
:10044000A1FE02F02FFF054602F074FF0446C0B97A
:100450000E4B9D4217D001339D4241F2883512BFA9
:10046000044600250124002002F026FF0CB100F014
:1004700075F800F027FE284600F01EF900F06EF82F
:10048000F9E70025EFE70546EDE700BF010007B0FB
:1004900008B500F073FCA0F120035842584108BD94
:1004A00007B541F21203022101A8ADF8043000F0B3
:1004B00083FC03B05DF804FB38B5302383F3118867
:1004C000174803680BB102F091FA0023154A4FF464
:1004D0007A71134802F080FA002383F31188124CDA
:1004E000236813B12368013B2360636813B1636819
:1004F000013B63600D4D2B7833B963687BB90220F3
:1005000000F042FD322363602B78032B07D1636830
:100510002BB9022000F038FD4FF47A73636038BDC8
:1005200070220020B90400089023002088220020B7
:10053000084B187003280CD8DFE800F00805020803
:10054000022000F013BD022000F000BD024B00228B
:100550005A6070478822002090230020F8B5504B45
:10056000504A1C461968013100F0998004339342C7
:10057000F8D162684C4B9A4240F291804B4B9B6899
:1005800003F1006303F500339A4280F08880002075
:1005900000F04EFC0220FFF7CBFF454B0021D3F8C3
:1005A000E820C3F8E810D3F81021C3F81011D3F8ED
:1005B0001021D3F8EC20C3F8EC10D3F81421C3F8C1
:1005C0001411D3F81421D3F8F020C3F8F010D3F8A5
:1005D0001821C3F81811D3F81821D3F8802042F05D
:1005E0000062C3F88020D3F8802022F00062C3F8B4
:1005F0008020D3F88020D3F8802042F00072C3F826
:100600008020D3F8802022F00072C3F88020D3F835
:10061000803072B64FF0E023C3F8084DD4E90004EF
:10062000BFF34F8FBFF36F8F224AC2F88410BFF31E
:100630004F8F536923F480335361BFF34F8FD2F848
:10064000803043F6E076C3F3C905C3F34E335B0154
:1006500003EA060C29464CEA81770139C2F8747224
:10066000F9D2203B13F1200FF2D1BFF34F8FBFF32C
:100670006F8FBFF34F8FBFF36F8F536923F4003336
:1006800053610023C2F85032BFF34F8FBFF36F8F17
:10069000302383F31188854680F308882047F8BD0E
:1006A0000000020820000208FFFF010800220020CD
:1006B0000044025800ED00E02DE9F04F93B0B44B38
:1006C0002022FF2100900AA89D6800F0A5FCB14AF5
:1006D0001378A3B90121B04811700360302383F36C
:1006E000118803680BB102F081F90023AB4A4FF483
:1006F0007A71A94802F070F9002383F31188009BF6
:1007000013B1A74B009A1A60A64A1378032B03D0A3
:1007100000231370A24A53604FF0000A009CD34696
:100720005646D146012000F021FC24B19C4B1B68A9
:10073000002B00F02682002000F020FB0390039B9A
:10074000002BF2DB012000F001FC039B213B1F2B5F
:10075000E8D801A252F823F0D907000801080008E0
:100760009508000825070008250700082507000848
:1007700027090008F70A0008110A0008730A000890
:100780009B0A0008C10A000825070008D30A0008D0
:1007900025070008450B0008790800082507000810
:1007A000890B0008E50700087908000825070008FC
:1007B000730A000825070008250700082507000818
:1007C0002507000825070008250700082507000859
:1007D00025070008950800080220FFF759FE0028A9
:1007E00040F0F981009B022105A8BAF1000F08BF73
:1007F0001C4641F21233ADF8143000F0DDFA91E7F7
:100800004FF47A7000F0BAFA071EEBDB0220FFF714
:100810003FFE0028E6D0013F052F00F2DE81DFE831
:1008200007F0030A0D1013360523042105A80593CC
:1008300000F0C2FA17E004215548F9E704215A48AC
:10084000F6E704215948F3E74FF01C08404608F149
:10085000040800F0EFFA0421059005A800F0ACFAB6
:10086000B8F12C0FF2D101204FF0000900FA07F780
:1008700047EA0B0B5FFA8BFB00F01AFC26B10BF07A
:100880000B030B2B08BF0024FFF70AFE4AE70421E5
:100890004748CDE7002EA5D00BF00B030B2BA1D1C1
:1008A0000220FFF7F5FD074600289BD00120002617
:1008B00000F0BEFA0220FFF73BFE1FFA86F8404622
:1008C00000F0C6FA0446B0B1039940460136A1F1E2
:1008D00040025142514100F0CBFA0028EDD1BA4616
:1008E000044641F21213022105A83E46ADF8143029
:1008F00000F062FA16E725460120FFF719FE244BA7
:100900009B68AB4207D9284600F094FA013040F0CA
:1009100067810435F3E70025224BBA463E461D7039
:100920001F4B5D60A8E7002E3FF45CAF0BF00B039C
:100930000B2B7FF457AF0220FFF7FAFD322000F0B7
:100940001DFAB0F10008FFF64DAF18F003077FF471
:1009500049AF0F4A08EB0503926893423FF642AF56
:10096000B8F5807F3FF73EAF124BB845019323DDCA
:100970004FF47A7000F002FA0390039A002AFFF60F
:1009800031AF039A0137019B03F8012BEDE700BF5C
:10099000002200208C23002070220020B9040008CF
:1009A000902300208822002004220020082200201A
:1009B0000C2200208C220020C820FFF769FD07468A
:1009C00000283FF40FAF1F2D11D8C5F120020AAB4C
:1009D00025F0030084494245184428BF424601924D
:1009E00000F0F4FA019AFF217F4800F015FB4FEA6E
:1009F000A803C8F387027C492846019300F014FB42
:100A0000064600283FF46DAF019B05EB830533E7F5
:100A10000220FFF73DFD00283FF4E4AE00F046FA67
:100A200000283FF4DFAE0027B846704B9B68BB42FE
:100A300018D91F2F11D80A9B01330ED027F00303BA
:100A400012AA134453F8203C05934046042205A9FA
:100A5000043700F0A9FB8046E7E7384600F0EAF9E2
:100A60000590F2E7CDF81480042105A800F0A4F960
:100A700002E70023642104A8049300F093F90028FE
:100A80007FF4B0AE0220FFF703FD00283FF4AAAECA
:100A9000049800F001FA0590E6E70023642104A819
:100AA000049300F07FF900287FF49CAE0220FFF74A
:100AB000EFFC00283FF496AE049800F0EFF9EAE767
:100AC0000220FFF7E5FC00283FF48CAE00F0FEF9B1
:100AD000E1E70220FFF7DCFC00283FF483AE05A924
:100AE000142000F0F9F907460421049004A800F04E
:100AF00063F93946B9E7322000F040F9071EFFF6E6
:100B000071AEBB077FF46EAE384A07EB09039268FB
:100B100093423FF667AE0220FFF7BAFC00283FF48D
:100B200061AE27F003074F44B9453FF4A5AE4846F0
:100B300009F1040900F07EF90421059005A800F0F0
:100B40003BF9F1E74FF47A70FFF7A2FC00283FF47D
:100B500049AE00F0ABF9002844D00A9B01330BD01A
:100B600008220AA9002000F05FFA00283AD02022CB
:100B7000FF210AA800F050FAFFF792FC1C4801F090
:100B800057FE13B0BDE8F08F002E3FF42BAE0BF0F4
:100B90000B030B2B7FF426AE0023642105A80593DD
:100BA00000F000F9074600287FF41CAE0220FFF792
:100BB0006FFC804600283FF415AEFFF771FC41F250
:100BC000883001F035FE059800F0BAFA46463C46FA
:100BD00000F06EFAA6E506464EE64FF0000901E683
:100BE000BA467EE637467CE68C22002000220020B2
:100BF000A08601002DE9F84F4FF47A7306460D46A2
:100C0000002402FB03F7DFF85080DFF8509098F9DA
:100C100000305FFA84FA5A1C01D0A34210D159F86F
:100C200024002A4631460368D3F820B03B46D84713
:100C3000854205D1074B012083F800A0BDE8F88F5D
:100C40000134042CE3D14FF4FA7001F0F1FD0020DF
:100C5000F4E700BFDC230020102200201422002033
:100C600000232DE9F0471A4605468846012019461B
:100C700000F09AFC0446802002F084FA074600281F
:100C800061D0002C5FD03B4E28464FF0800A73693C
:100C900043F0C0637361D6F8143143F0C063C6F803
:100CA000143102F0F3F805EB080200FB05F34FF4F2
:100CB000D06C50434FF03D0E834233D23269520123
:100CC00043D4D6F8102151013FD4216803F10062CA
:100CD0008A602268D7602268C2F804A02268C2F83D
:100CE00000C0D4F80090D9F8002042F00102C9F801
:100CF0000020D4F80090D9F8002022F01E02C9F894
:100D00000020D4F80090D9F80020D207FBD494F842
:100D10000C90803361680EFA09F20A60CCE700207B
:100D200002F092F9204600F07FFC384602F064FAA7
:100D3000104B5A6942F0C0625A61D3F8142142F054
:100D4000C062C3F81421BDE8F0870B4B9A6A42F4E5
:100D500000729A629A6A42F400429A6261B6002670
:100D6000012002F071F9B045D9D9A819013602F075
:100D7000A5F8F8E70020005200ED00E0002307B5D9
:100D8000024601210DF107008DF80730FFF732FF11
:100D900020B19DF8070003B05DF804FB4FF0FF3071
:100DA000F9E700000A46042108B5FFF723FF80F0A9
:100DB0000100C0B2404208BD074B0A4630B4197862
:100DC000064B53F82140014623682046DD69044B59
:100DD000AC4630BC604700BFDC230020142200205A
:100DE000A086010070B5104C0025104E02F052F89C
:100DF00020803068238883420CD800252088013861
:100E000002F044F823880544013BB5F5802F238088
:100E1000F4D370BD02F03AF8336805440133B5F5F8
:100E2000003F3360E5D3E8E7DE230020982300206D
:100E300002F00AB900F1006000F500300068704768
:100E400000F10060920000F5003002F07FB8000071
:100E5000054B1A68054B1B889B1A834202D9104424
:100E600002F014B80020704798230020DE230020F1
:100E700038B50446074D29B128682044BDE83840FC
:100E800002F01CB82868204402F006F80028F3D0CD
:100E900038BD00BF982300200020704700F1FF50AC
:100EA00000F58F10D0F8000870470000064991F84F
:100EB000243033B100230822086A81F82430FFF778
:100EC000BFBF0120704700BF9C230020014B186862
:100ED000704700BF0010005C194B01380322084422
:100EE00070B51D68174BC5F30B042D0C1E88A64268
:100EF0000BD15C680A46013C824213460FD214F9BA
:100F0000016F4EB102F8016BF6E7013A03F10803F5
:100F1000ECD181420B4602D22C2203F8012B04248F
:100F2000094A1688AE4204D1984284BF967803F8E5
:100F3000016B013C02F10402F3D1581A70BD00BFED
:100F40000010005C24220020A8590008022804D1C7
:100F5000054B4FF400129A6170470128FCD1024BF7
:100F60004FF40022F7E700BF00100258022803D117
:100F7000044B20229A6170470128FCD1014B0822C2
:100F8000F8E700BF00100258022805D1064A53694D
:100F900083F02003536170470128FCD1024A536952
:100FA00083F00803F6E700BF0010025870B504464E
:100FB0004FF47A764CB1412C254628BF412506FBDB
:100FC00005F0641B01F034FCF4E770BD002310B59C
:100FD000934203D0CC5CC4540133F9E710BD000048
:100FE000013810B510F9013F3BB191F900409C4226
:100FF00003D11AB10131013AF4E71AB191F9002095
:10100000981A10BD1046FCE703460246D01A12F9A2
:10101000011B0029FAD1704702440346934202D0D3
:1010200003F8011BFAE770472DE9F8431F4D1446FA
:101030000746884695F8242052BBDFF870909CB391
:1010400095F824302BB92022FF2148462F62FFF764
:10105000E3FF95F824004146C0F1080205EB80004B
:10106000A24228BF2246D6B29200FFF7AFFF95F802
:101070002430A41B17441E449044E4B2F6B2082E58
:1010800085F82460DBD1FFF711FF0028D7D108E0F5
:101090002B6A03EB82038342CFD0FFF707FF0028C0
:1010A000CBD10020BDE8F8830120FBE79C23002082
:1010B000024B1A78024B1A70704700BFDC230020E5
:1010C00010220020F8B5194C194800F0E1FE214625
:1010D000174800F009FF24684FF47A70154ED4F8D1
:1010E0009020154DD2F80438114F43F00203C2F896
:1010F0000438FFF75BFF2046104901F003F8D4F8ED
:1011000090200424D2F8043823F00203C2F80438F3
:101110004FF4E133336055F8040BB84202D0314646
:1011200000F014FE013CF6D1F8BD00BFA45B00083E
:1011300088380020C423002014220020AC5B000863
:101140000C4B70B50C4D04461E780C4B55F8262000
:101150009A420DD00A4B002118221846FFF75CFF77
:101160000460014655F82600BDE8704000F0EEBD71
:1011700070BD00BFDC23002014220020883800202E
:10118000C423002008B571B6054B1988054B188893
:10119000FFF766FD02210E20FFF762FD61B608BD74
:1011A000DE2300209823002030B50A44084D9142E8
:1011B0000DD011F8013B5840082340F30004013BD7
:1011C0002C4013F0FF0384EA5000F6D1EFE730BD66
:1011D0002083B8ED08B5074B074A196801F03D01B7
:1011E000996053680BB190689847BDE8084002F0D9
:1011F000E3B800BF00000240E023002008B5084B20
:101200001968890901F03D018A019A60054AD3688D
:101210000BB110699847BDE8084002F0CDB800BF97
:1012200000000240E023002008B5084B1968090CB3
:1012300001F03D010A049A60054A53690BB19069B7
:101240009847BDE8084002F0B7B800BF0000024070
:10125000E023002008B5084B1968890D01F03D0115
:101260008A059A60054AD3690BB1106A9847BDE8B0
:10127000084002F0A1B800BF00000240E0230020B7
:1012800008B5074B074A596801F03D01D960536A18
:101290000BB1906A9847BDE8084002F08DB800BFD6
:1012A00000000240E023002008B5084B5968890976
:1012B00001F03D018A01DA60054AD36A0BB1106B77
:1012C0009847BDE8084002F077B800BF0000024030
:1012D000E023002008B5084B5968090C01F03D01D6
:1012E0000A04DA60054A536B0BB1906B9847BDE86E
:1012F000084002F061B800BF00000240E023002077
:1013000008B5084B5968890D01F03D018A05DA607E
:10131000054AD36B0BB1106C9847BDE8084002F04A
:101320004BB800BF00000240E023002008B5074B87
:10133000074A196801F03D019960536C0BB1906C3C
:101340009847BDE8084002F037B800BF00040240EB
:10135000E023002008B5084B1968890901F03D0118
:101360008A019A60054AD36C0BB1106D9847BDE8AD
:10137000084002F021B800BF00040240E023002032
:1013800008B5084B1968090C01F03D010A049A6080
:10139000054A536D0BB1906D9847BDE8084002F0C7
:1013A0000BB800BF00040240E023002008B5084B42
:1013B0001968890D01F03D018A059A60054AD36DCF
:1013C0000BB1106E9847BDE8084001F0F5BF00BFB3
:1013D00000040240E023002008B5074B074A596883
:1013E00001F03D01D960536E0BB1906E9847BDE896
:1013F000084001F0E1BF00BF00040240E0230020EC
:1014000008B5084B5968890901F03D018A01DA6085
:10141000054AD36E0BB1106F9847BDE8084001F044
:10142000CBBF00BF00040240E023002008B5084BFA
:101430005968090C01F03D010A04DA60054A536F4E
:101440000BB1906F9847BDE8084001F0B5BF00BFF1
:1014500000040240E023002008B5084B5968890DBC
:1014600001F03D018A05DA60054AD36F13B1D2F865
:1014700080009847BDE8084001F09EBF000402408C
:10148000E023002000230C4910B51A460B4C0B60DA
:1014900054F82300026001EB430004334260402B08
:1014A000F6D1074A4FF0FF339360D360C2F8083497
:1014B000C2F80C3410BD00BFE0230020B85900086A
:1014C000000002400F28F8B510D9102810D01128BC
:1014D00011D0122808D10F240720DFF8C8E0012618
:1014E000DEF80050A04208D9002653E00446F4E795
:1014F0000F240020F1E70724FBE706FA00F73D423E
:101500004AD1264C4FEA001C3D4304EB00160EEB7B
:10151000C000CEF80050C0E90123FBB273B12048EF
:10152000D0F8D83043F00103C0F8D830D0F80031FB
:1015300043F00103C0F80031D0F8003117F47F4FB9
:101540000ED01748D0F8D83043F00203C0F8D83096
:10155000D0F8003143F00203C0F80031D0F8003178
:1015600054F80C00036823F01F030360056815F0AE
:101570000105FBD104EB0C033D2493F80CC05F681C
:1015800004FA0CF43C6021240560446112B1987B9C
:1015900000F010FA3046F8BD0130A3E7B859000852
:1015A00000440258E023002010B5302484F3118851
:1015B000FFF788FF002383F3118810BD10B50446A0
:1015C000807B00F00DFA01231549627B03FA02F2D9
:1015D0000B6823EA0203DAB20B6072B9114AD2F83F
:1015E000D81021F00101C2F8D810D2F8001121F072
:1015F0000101C2F80011D2F8002113F47F4F0ED17F
:10160000084BD3F8D82022F00202C3F8D820D3F830
:10161000002122F00202C3F80021D3F8003110BDEE
:10162000E02300200044025808B5302383F31188DA
:10163000FFF7C4FF002383F3118808BD02684368E5
:101640001143016003B1184770470000024A136854
:1016500043F0C0031360704700100140024A136852
:1016600043F0C0031360704700480040024A13680B
:1016700043F0C0031360704700500040024A1368F3
:1016800043F0C0031360704700780040064BD3F866
:10169000E8200243C3F8E820D3F810211043C3F830
:1016A0001001D3F8103170470044025837B5334C5D
:1016B000334D204600F03EFB04F11400009400235B
:1016C0004FF400722F4900F0FBF94FF400722E49DD
:1016D00004F1380000942D4B00F074FA2C4BC4E94F
:1016E00017352C4C204600F025FB04F11400009423
:1016F00000234FF40072284900F0E2F94FF4007221
:10170000264904F138000094254B00F05BFA254B84
:10171000C4E91735244C204600F00CFB04F11400FA
:10172000009400234FF40072204900F0C9F94FF4EF
:1017300000721F4904F1380000941E4B00F042FA79
:101740001D4BC4E917351D4C204600F0F3FA04F197
:10175000140000234FF400721949009400F0B0F90E
:10176000184B4FF40072184904F13800009400F04F
:1017700029FA164BC4E9173503B030BD64240020A4
:1017800000E1F50514260020142E00204D16000857
:1017900000100140D0240020142800201430002024
:1017A0005D160008004800403C250020142A002057
:1017B000143200206D16000800500040A8250020BB
:1017C000142C00207D1600081434002000780040FE
:1017D00038B52F4D0446037C002918BF0D46012B58
:1017E00011D12C4B98423BD12B4BD3F8F02042F037
:1017F0001002C3F8F020D3F8182142F01002C3F809
:101800001821D3F818312A68236EE16D03EB5203D7
:10181000A566B3FBF2F36A68100442BF23F0070029
:1018200003F0070343EA4003CB60AB6843F0400397
:101830004B60EB6843F001038B6042F4967343F016
:1018400001030B604FF0FF330B62510505D512F019
:10185000102219D0B2F1805F18D084F8643038BDFE
:101860000E4B984205D00E4B984207D14FF4801092
:1018700001E04FF48020FFF709FFC4E7094B9842CD
:10188000C1D14FF08040F6E77F23E6E73F23E4E74E
:10189000B85A00086424002000440258D0240020D4
:1018A0003C250020A82500202DE9F047C66D0546FF
:1018B0003768F469210734621AD014F0080118BFA0
:1018C0004FF48071E20748BF41F02001A3074FF0B9
:1018D000300348BF41F04001600748BF41F080013C
:1018E00083F31188281DFFF7A9FE002383F31188D5
:1018F000E2050AD5302383F311884FF48061281D57
:10190000FFF79CFE002383F311884FF030094FF05E
:10191000000A14F0200838D13B0616D54FF03009E4
:1019200005F1380A200610D589F31188504600F0D9
:101930007DF9002836DA0821281DFFF77FFE27F001
:1019400080033360002383F31188790614D562067F
:1019500012D5302383F31188D5E913239A4208D195
:101960002B6C33B127F040071021281DFFF766FECE
:101970003760002383F31188E30618D5AA6E136934
:10198000ABB15069BDE8F047184789F31188736A15
:10199000284695F86410194000F0E6F98AF311889A
:1019A000F469B6E7B06288F31188F469BAE7BDE874
:1019B000F0870000090100F16043012203F5614353
:1019C000C9B283F8001300F01F039A4043099B003B
:1019D00003F1604303F56143C3F880211A60704747
:1019E00000F01F0301229A40430900F160409B0070
:1019F00000F5614003F1604303F56143C3F88020C3
:101A0000C3F88021002380F800337047F8B51546ED
:101A1000826804460B46AA4200D28568A1692669FD
:101A2000761AB5420BD218462A46FFF7CFFAA369B9
:101A30002B44A3612846A3685B1BA360F8BD0CD9A7
:101A4000AF1B18463246FFF7C1FA3A46E168304408
:101A5000FFF7BCFAE3683B44EBE718462A46FFF77A
:101A6000B5FAE368E5E7000083689342F7B50446FA
:101A7000154600D28568D4E90460361AB5420BD207
:101A80002A46FFF7A3FA63692B4463612846A368DB
:101A90005B1BA36003B0F0BD0DD93246AF1B0191B3
:101AA000FFF794FA01993A46E0683144FFF78EFA5D
:101AB000E3683B44E9E72A46FFF788FAE368E4E78E
:101AC00010B50A440024C361029B8460C1600261B6
:101AD0000362C0E90000C0E9051110BD08B5D0E9F6
:101AE0000532934201D1826882B9826801328260F4
:101AF0005A1C426119700021D0E904329A4224BF75
:101B0000C368436100F0C8FE002008BD4FF0FF30FD
:101B1000FBE7000070B5302304460E4683F31188BE
:101B2000A568A5B1A368A269013BA360531CA3618A
:101B300015782269934224BFE368A361E3690BB17E
:101B400020469847002383F31188284607E0314652
:101B5000204600F091FE0028E2DA85F3118870BD7E
:101B60002DE9F74F04460E4617469846D0F81C90CC
:101B70004FF0300A8AF311884FF0000B154665B11B
:101B80002A4631462046FFF741FF034660B94146E9
:101B9000204600F071FE0028F1D0002383F3118865
:101BA000781B03B0BDE8F08FB9F1000F03D00190AE
:101BB0002046C847019B8BF31188ED1A1E448AF317
:101BC0001188DCE7C160C361009B82600362C0E9E9
:101BD00005111144C0E9000001617047F8B50446E1
:101BE0000D461646302383F31188A768A7B1A36872
:101BF000013BA36063695A1C62611D70D4E9043221
:101C00009A4224BFE3686361E3690BB120469847B9
:101C1000002080F3118807E03146204600F02CFEBA
:101C20000028E2DA87F31188F8BD0000D0E9052327
:101C300010B59A4201D182687AB9826800210132D6
:101C400082605A1C82611C7803699A4224BFC3686F
:101C5000836100F021FE204610BD4FF0FF30FBE70E
:101C60002DE9F74F04460E4617469846D0F81C90CB
:101C70004FF0300A8AF311884FF0000B154665B11A
:101C80002A4631462046FFF7EFFE034660B941463B
:101C9000204600F0F1FD0028F1D0002383F31188E5
:101CA000781B03B0BDE8F08FB9F1000F03D00190AD
:101CB0002046C847019B8BF31188ED1A1E448AF316
:101CC0001188DCE7026843681143016003B11847DB
:101CD000704700001430FFF743BF00004FF0FF33A0
:101CE0001430FFF73DBF00003830FFF7B9BF0000E8
:101CF0004FF0FF333830FFF7B3BF00001430FFF769
:101D000009BF00004FF0FF311430FFF703BF0000A0
:101D10003830FFF763BF00004FF0FF323830FFF775
:101D20005DBF0000012914BF6FF013000020704751
:101D3000FFF7BCBC044B036000234360C0E90233DF
:101D400001230374704700BFD05A000810B5302338
:101D5000044683F31188FFF73BFD02230020237420
:101D600080F3118810BD000038B5C36904460D46E4
:101D70001BB904210844FFF7A5FF294604F114000C
:101D8000FFF7ACFE002806DA201D4FF40061BDE825
:101D90003840FFF797BF38BD0268436811430160C0
:101DA00003B118477047000013B5406B00F580542D
:101DB000D4F8A4381A681178042914D1017C0229B6
:101DC00011D11979012312898B4013420BD101A93A
:101DD0004C3002F0E1F9D4F8A4480246019B217985
:101DE000206800F0DFF902B010BD0000143002F0EE
:101DF00063B900004FF0FF33143002F05DB900000A
:101E00004C3002F035BA00004FF0FF334C3002F096
:101E10002FBA0000143002F031B900004FF0FF314A
:101E2000143002F02BB900004C3002F001BA00006F
:101E30004FF0FF324C3002F0FBB900000020704739
:101E400010B500F58054D4F8A4381A681178042924
:101E500017D1017C022914D15979012352898B4071
:101E600013420ED1143002F0C3F8024648B1D4F840
:101E7000A4484FF4407361792068BDE8104000F039
:101E80007FB910BD406BFFF7DBBF0000704700005B
:101E90007FB5124B01250426044603600023057418
:101EA00000F1840243602946C0E902330C4B0290E2
:101EB000143001934FF44073009602F075F8094B0B
:101EC00004F69442294604F14C000294CDE90063E3
:101ED0004FF4407302F03CF904B070BDF85A0008AA
:101EE000851E0008A91D00080A68302383F31188A5
:101EF0000B790B3342F823004B79133342F823005C
:101F00008B7913B10B3342F8230000F58053C3F8EB
:101F1000A41802230374002080F311887047000086
:101F200038B5037F044613B190F85430ABB901259E
:101F3000201D0221FFF730FF04F114006FF00101B2
:101F4000257700F0B5FC04F14C0084F854506FF094
:101F50000101BDE8384000F0ABBC38BD10B501212F
:101F600004460430FFF718FF0023237784F8543029
:101F700010BD000038B504460025143002F02CF8DE
:101F800004F14C00257702F0FBF8201D84F8545032
:101F90000121FFF701FF2046BDE83840FFF750BFA1
:101FA00090F8803003F06003202B06D190F8812058
:101FB0000023212A03D81F2A06D800207047222A8E
:101FC000FBD1C0E91D3303E0034A42670722826761
:101FD000C3670120704700BF3C22002037B500F5E1
:101FE0008055D5F8A4381A68117804291AD1017CD3
:101FF000022917D11979012312898B40134211D17B
:1020000000F14C04204602F07BF958B101A92046AA
:1020100002F0C2F8D5F8A4480246019B2179206855
:1020200000F0C0F803B030BD01F10B03F0B550F87B
:10203000236085B004460D46FEB1302383F311883A
:1020400004EB8507301D0821FFF7A6FEFB6806F1AB
:102050004C005B691B681BB1019002F0ABF8019862
:1020600003A902F099F8024648B1039B294620468D
:1020700000F098F8002383F3118805B0F0BDFB68E9
:102080005A691268002AF5D01B8A013B1340F1D12E
:1020900004F18002EAE70000133138B550F821401E
:1020A000ECB1302383F3118804F58053D3F8A428CE
:1020B0001368527903EB8203DB689B695D6845B165
:1020C00004216018FFF768FE294604F1140001F0AE
:1020D00099FF2046FFF7B4FE002383F3118838BD33
:1020E0007047000001F066BA01234022002110B5BC
:1020F000044600F8303BFEF78FFF0023C4E90133AC
:1021000010BD000010B53023044683F3118824224B
:10211000416000210C30FEF77FFF204601F06CFA91
:1021200002230020237080F3118810BD70B500EBEE
:102130008103054650690E461446DA6018B1102234
:102140000021FEF769FFA06918B110220021FEF7F7
:1021500063FF31462846BDE8704001F053BB0000E4
:1021600083682022002103F0011310B50446836028
:102170001030FEF751FF2046BDE8104001F0CEBB05
:10218000F0B4012500EB810447898D40E4683D43AC
:10219000A469458123600023A2606360F0BC01F064
:1021A000EBBB0000F0B4012500EB810407898D40F2
:1021B000E4683D436469058123600023A260636095
:1021C000F0BC01F061BC000070B50223002504469C
:1021D000242203702946C0F888500C3040F8045C73
:1021E000FEF71AFF204684F8705001F09FFA6368EA
:1021F0001B6823B129462046BDE87040184770BDD2
:102200000378052B10B504460AD080F88C300523DE
:10221000037043681B680BB1042198470023A36037
:1022200010BD00000178052906D190F88C20436884
:1022300002701B6803B118477047000070B590F832
:102240007030044613B1002380F8703004F180022E
:10225000204601F087FB63689B68B3B994F880302F
:1022600013F0600535D00021204601F079FE0021F1
:10227000204601F069FE63681B6813B10621204601
:102280009847062384F8703070BD20469847002890
:10229000E4D0B4F88630A26F9A4288BFA36794F95D
:1022A0008030A56F002B4FF0300380F20381002DAA
:1022B00000F0F280092284F8702083F31188002155
:1022C0002046D4E91D23FFF76DFF002383F3118817
:1022D000DAE794F8812003F07F0343EA022340F217
:1022E0000232934200F0C58021D8B3F5807F48D0F8
:1022F0000DD8012B3FD0022B00F09380002BB2D1E0
:1023000004F1880262670222A267E367C1E7B3F5BE
:10231000817F00F09B80B3F5407FA4D194F8823098
:10232000012BA0D1B4F8883043F0020332E0B3F5BA
:10233000006F4DD017D8B3F5A06F31D0A3F5C063AF
:10234000012B90D86368204694F882205E6894F848
:102350008310B4F88430B047002884D043686367A2
:102360000368A3671AE0B3F5106F36D040F6024257
:1023700093427FF478AF5C4B63670223A36700232B
:10238000C3E794F88230012B7FF46DAFB4F8883046
:1023900023F00203A4F88830C4E91D55E56778E707
:1023A000B4F88030B3F5A06F0ED194F88230204697
:1023B00084F88A3001F018FA63681B6813B10121B0
:1023C00020469847032323700023C4E91D339CE76C
:1023D00004F18B0363670123C3E72378042B10D137
:1023E000302383F311882046FFF7BAFE85F3118866
:1023F0000321636884F88B5021701B680BB1204661
:10240000984794F88230002BDED084F88B30042378
:10241000237063681B68002BD6D0022120469847A2
:10242000D2E794F8843020461D0603F00F010AD548
:1024300001F08AFA012804D002287FF414AF2B4B54
:102440009AE72B4B98E701F071FAF3E794F88230A2
:10245000002B7FF408AF94F8843013F00F01B3D051
:102460001A06204602D501F093FDADE701F084FD88
:10247000AAE794F88230002B7FF4F5AE94F884300C
:1024800013F00F01A0D01B06204602D501F068FD15
:102490009AE701F059FD97E7142284F8702083F33E
:1024A00011882B462A4629462046FFF769FE85F308
:1024B0001188E9E65DB1152284F8702083F3118854
:1024C00000212046D4E91D23FFF75AFEFDE60B222A
:1024D00084F8702083F311882B462A46294620462B
:1024E000FFF760FEE3E700BF285B0008205B000801
:1024F000245B000838B590F870300446002B3ED0BD
:10250000063BDAB20F2A34D80F2B32D8DFE803F0BB
:1025100037313108223231313131313131313737D0
:10252000856FB0F886309D4214D2C3681B8AB5FB14
:10253000F3F203FB12556DB9302383F311882B4658
:102540002A462946FFF72EFE85F311880A2384F8D0
:1025500070300EE0142384F87030302383F3118838
:10256000002320461A461946FFF70AFE002383F38C
:10257000118838BDC36F03B198470023E7E70021F6
:10258000204601F0EDFC0021204601F0DDFC6368EF
:102590001B6813B10621204698470623D7E70000A1
:1025A00010B590F870300446142B29D017D8062B9C
:1025B00005D001D81BB110BD093B022BFBD800216F
:1025C000204601F0CDFC0021204601F0BDFC6368EF
:1025D0001B6813B1062120469847062319E0152BE6
:1025E000E9D10B2380F87030302383F31188002366
:1025F0001A461946FFF7D6FD002383F31188DAE760
:10260000C3689B695B68002BD5D1C36F03B1984742
:10261000002384F87030CEE70023826803750369D5
:102620001B6899689142FBD25A680360426010604F
:102630005860704700238268037503691B689968B6
:102640009142FBD85A68036042601060586070473E
:1026500008B50846302383F311880A7D0023052A34
:1026600006D8DFE802F00B050503120E826913603D
:102670004FF0FF338361FFF7CFFF002383F311880F
:1026800008BD8269936801339360D0E9003213601A
:102690005A60EDE7FFF7C0BF054BD96808751868A9
:1026A000026853601A600122D8600275FDF7AABE65
:1026B000183600200C4B30B5DD684B1C87B0044643
:1026C0000FD02B46094A684600F086F92046FFF7EE
:1026D000E3FF009B13B1684600F088F9A86907B0D2
:1026E00030BDFFF7D9FFF9E7183600205126000862
:1026F00038B50C4D04468161EB6881689A68914257
:1027000003D8BDE83840FFF787BF1846FFF792FFB0
:1027100001230146EC6020462375BDE83840FDF7F3
:1027200071BE00BF18360020044B1A68DB68906841
:102730009B68984294BF0020012070471836002003
:10274000084B10B51C68D868226853601A600122D3
:10275000DC602275FFF76EFF01462046BDE81040A1
:10276000FDF750BE1836002038B50123084C00256F
:102770002370656001F000FE01F026FE0549064861
:1027800001F0FAFE0223237085F3118838BD00BFE3
:1027900080380020305B00081836002000F05CB95B
:1027A000034A516853685B1A9842FBD8704700BFD0
:1027B000001000E08B600223086108468B8270479E
:1027C0008368A3F1840243F8142C026943F8442C73
:1027D000426943F8402C094A43F8242CC268A3F10B
:1027E000200043F8182C022203F80C2C002203F8D6
:1027F0000B2C034A43F8102C704700BF1D0400083F
:102800001836002008B5FFF7DBFFBDE80840FFF7EA
:1028100041BF0000024BDB6898610F20FFF73CBF0F
:1028200018360020302383F31188FFF7F3BF000030
:1028300008B50146302383F311880820FFF73AFFDB
:10284000002383F3118808BD054BDB6821B10360C9
:1028500098610320FFF72EBF4FF0FF30704700BF95
:102860001836002003682BB10022026018469961D7
:10287000FFF710BF70470000064BDB6839B14268B4
:1028800018605A60136043600420FFF713BF4FF0D5
:10289000FF307047183600200368984206D01A6847
:1028A0000260506018469961FFF7F4BE704700005F
:1028B00038B504460D462068844200D138BD03680F
:1028C00023605C608561FFF7E5FEF4E7036810B5FF
:1028D0009C68A2420CD85C688A600B604C602160E6
:1028E000596099688A1A9A604FF0FF33836010BD6F
:1028F000121B1B68ECE700000A2938BF0A2170B5DB
:1029000004460D460A26601901F030FD01F018FD5D
:10291000041BA54203D8751C04462E46F3E70A2E75
:1029200004D90120BDE8704001F066BE70BD000012
:10293000F8B5144B0D460A2A4FF00A07D96103F186
:102940001001826038BF0A22416019691446016093
:1029500048601861A81801F0F9FC01F0F1FC431B74
:102960000646A34206D37C1C28192746354601F0AB
:10297000FDFCF2E70A2F04D90120BDE8F84001F080
:102980003BBEF8BD18360020F8B506460D4601F0EE
:10299000D7FC0F4A134653F8107F9F4206D12A46B0
:1029A00001463046BDE8F840FFF7C2BFD169BB68B9
:1029B000441A2C1928BF2C46A34202D92946FFF7F6
:1029C0009BFF224631460348BDE8F840FFF77EBF33
:1029D0001836002028360020C0E90323002310B455
:1029E0005DF8044B4361FFF7CFBF000010B5194CF1
:1029F000236998420DD08168D0E9003213605A6093
:102A00009A680A449A60002303604FF0FF33A36181
:102A100010BD0268234643F8102F53600022026065
:102A200022699A4203D1BDE8104001F099BC936835
:102A300081680B44936001F083FC2269E16992682C
:102A4000441AA242E4D91144BDE81040091AFFF724
:102A500053BF00BF183600202DE9F047DFF8BC80D7
:102A600008F110072C4ED8F8105001F069FCD8F886
:102A70001C40AA68031B9A423ED814444FF0000938
:102A8000D5E90032C8F81C4013605A60C5F80090C0
:102A9000D8F81030B34201D101F062FC89F31188FB
:102AA000D5E9033128469847302383F311886B69B1
:102AB000002BD8D001F044FC6A69A0EB04098246DF
:102AC0004A450DD2022001F097FD0022D8F81030BF
:102AD000B34208D151462846BDE8F047FFF728BF6A
:102AE000121A2244F2E712EB09092946384638BF88
:102AF0004A46FFF7EBFEB5E7D8F81030B34208D0EE
:102B00001444C8F81C00211AA960BDE8F047FFF77B
:102B1000F3BEBDE8F08700BF28360020183600203D
:102B200000207047FEE70000704700004FF0FF30C4
:102B30007047000002290CD0032904D0012907485E
:102B400018BF00207047032A05D8054800EBC200D3
:102B50007047044870470020704700BF085C0008B9
:102B60004C220020BC5B000870B59AB005460846B0
:102B7000144601A900F0C2F801A8FEF745FA431C6B
:102B80000022C6B25B001046C5E90034237003235F
:102B9000023404F8013C01ABD1B202348E4201D8B8
:102BA0001AB070BD13F8011B013204F8010C04F8CF
:102BB000021CF1E708B5302383F311880348FFF7BF
:102BC0000DFA002383F3118808BD00BF8838002068
:102BD00090F8803003F01F02012A07D190F881207D
:102BE0000B2A03D10023C0E91D3315E003F0600375
:102BF000202B08D1B0F884302BB990F88120212AFD
:102C000003D81F2A04D8FFF7CBB9222AEBD0FAE762
:102C1000034A426707228267C3670120704700BFEB
:102C20004322002007B5052917D8DFE801F019165F
:102C300003191920302383F31188104A01210190D0
:102C4000FFF774FA019802210D4AFFF76FFA0D4859
:102C5000FFF790F9002383F3118803B05DF804FBBC
:102C6000302383F311880748FFF75AF9F2E730233E
:102C700083F311880348FFF771F9EBE75C5B000809
:102C8000805B00088838002038B50C4D0C4C2A4673
:102C90000C4904F10800FFF767FF05F1CA0204F1CF
:102CA00010000949FFF760FF05F5CA7204F118002A
:102CB0000649BDE83840FFF757BF00BF605100200C
:102CC0004C2200203C5B0008465B0008515B00087A
:102CD00070B5044608460D46FEF796F9C6B2204682
:102CE000013403780BB9184670BD32462946FEF709
:102CF00077F90028F3D10120F6E700002DE9F84F1D
:102D000005460C46FEF780F92A49C6B22846FFF769
:102D1000DFFF08B10136F6B227492846FFF7D8FF92
:102D200008B11036F6B2632E0DD8DFF88890DFF8C0
:102D300088A0224FDFF88CB0DFF88C802E7846B95F
:102D40002670BDE8F88F29462046BDE8F84F02F00E
:102D50000DBE252E2AD1072249462846FEF740F906
:102D600050B9D8F800300735083444F8083CD8F892
:102D7000043044F8043CE1E7082251462846FEF7B7
:102D80002FF998B9A21C0E4B197802320909C95DB6
:102D900002F8041C13F8011B01F00F015B45C95D2B
:102DA00002F8031CF0D118340835C7E7013504F8E0
:102DB000016BC3E7285C0008515B0008395C000820
:102DC00000E8F11F0CE8F11F305C0008BFF34F8FE3
:102DD000044B1A695107FCD1D3F810215207F8D1DE
:102DE000704700BF0020005208B50D4B1B78ABB9EF
:102DF000FFF7ECFF0B4BDA68D10704D50A4A5A609B
:102E000002F188325A60D3F80C21D20706D5064A5F
:102E1000C3F8042102F18832C3F8042108BD00BFC1
:102E2000BE530020002000522301674508B5114B16
:102E30001B78F3B9104B1A69510703D5DA6842F0D1
:102E40004002DA60D3F81021520705D5D3F80C21DF
:102E500042F04002C3F80C21FFF7B8FF064BDA68D6
:102E600042F00102DA60D3F80C2142F00102C3F80B
:102E70000C2108BDBE530020002000520F289ABF2D
:102E800000F5806040040020704700004FF40030DF
:102E900070470000102070470F2808B50BD8FFF7C7
:102EA000EDFF00F500330268013204D104308342A3
:102EB000F9D1012008BD0020FCE700000F2838B53B
:102EC00005463FD8FFF782FF1F4CFFF78DFF4FF0FD
:102ED000FF3307286361C4F814311DD82361FFF75D
:102EE00075FF030243F02403E360E36843F08003CB
:102EF000E36023695A07FCD42846FFF767FFFFF712
:102F0000BDFF4FF4003100F0E5F92846FFF78EFFD2
:102F1000BDE83840FFF7C0BFC4F81031FFF756FFD7
:102F2000A0F108031B0243F02403C4F80C31D4F8C9
:102F30000C3143F08003C4F80C31D4F810315B0736
:102F4000FBD4D9E7002038BD002000522DE9F84F0E
:102F500004460D46104644EA0203DE0602D0002075
:102F6000BDE8F88F20F01F00DFF8D4B0DFF8D4A060
:102F7000FFF73AFF05EB0008454503D10120FFF7B5
:102F800055FFEDE720222946204602F0DFFC10B96C
:102F900020342035F0E7234604F120021F68791C15
:102FA000DDD104339342F9D104F178432048214E16
:102FB000B3F5801F204B38BF184603F1F80332BF2A
:102FC000D946D1461E46FFF701FF0760A4EB050C6A
:102FD000336805F11C0143F0020333602B1FD9F85D
:102FE000007017F00507FAD153F8042F8B424CF804
:102FF0000320F4D1BFF34F8FFFF7E8FE4FF0FF330C
:103000000360336823F002033360BFF34F8F0B4B31
:10301000C3F85C42BFF34F8FBFF36F8F2022294666
:10302000204602F093FC0028B2D03846A7E700BF44
:10303000142100520C2000521420005200ED00E038
:10304000102000521021005210B5084C237828B1EE
:103050001BB9FFF7C9FE0123237010BD002BFCD064
:103060002070BDE81040FFF7E1BE00BFBE53002056
:103070002DE9F04F0D4685B0814658B111F00D068F
:1030800014BF2022082211F00803019304D0431E2C
:1030900003426AD0002435E0002E37D009F11F0129
:1030A00021F01F094FF00108324F05F00403DFF84B
:1030B000D0A005EA080BBBF1000F32D07869C00739
:1030C0002FD408F101080C37B8F1060FF3D19EB9DF
:1030D000294D4946A819019201F098F904460028A3
:1030E0003AD11836019A782EF3D1494601F08EF97B
:1030F0000446002830D1019A4946204801F086F95B
:10310000044668BB204605B0BDE8F08F0029C9D150
:1031100001462846029201F079F90446E0B9029A84
:10312000C0E713B178694107CBD5AC0702D5786900
:103130008007C6D5019911B178690107C1D518205A
:10314000494600FB08A0CDE9022301F05FF90446DF
:10315000DDE902230028B4D04A460021204601E0E0
:103160004A460021FDF758FFCCE70246002E95D1D4
:1031700098E700BF4C5C0008F0530020C0530020CB
:10318000D85300200121FFF773BF0000F8B50023DA
:103190001A461A600433B3F5806FFAD1114D012439
:1031A0001827114E07FB046001342A6955F80C1FDB
:1031B00001F018F9062CF5D137254FF4C0542046FC
:1031C000FFF7E0FF014628B122460848BDE8F84075
:1031D00001F008B9C4EBC404013D4FEAD404EED1B8
:1031E000F8BD00BF4C5C0008D8530020C05300203D
:1031F0000421FFF73DBF000008B101F079B9704725
:1032000070B5AAB140EA010313F01F030FD1094CB6
:103210000144A5686D0706D52568A84203D36668F2
:103220003544A94204D903330C34122BF1D10022C6
:10323000104670BD4C5C00080244074BD2B210B57A
:10324000904200D110BD441C00B253F8200041F858
:10325000040BE0B2F4E700BF504000580E4B30B50D
:103260001C6F240405D41C6F1C671C6F44F40044BD
:103270001C670A4C02442368D2B243F48073236073
:10328000074B904200D130BD441C51F8045B00B2A2
:1032900043F82050E0B2F4E70044025800480258D6
:1032A0005040005807B5012201A90020FFF7C4FFD4
:1032B000019803B05DF804FB13B50446FFF7F2FF75
:1032C000A04205D0012201A900200194FFF7C6FF0A
:1032D00002B010BD0144BFF34F8F064B884204D3A8
:1032E000BFF34F8FBFF36F8F7047C3F85C0220307E
:1032F000F4E700BF00ED00E00144BFF34F8F064B41
:10330000884204D3BFF34F8FBFF36F8F7047C3F86A
:1033100070022030F4E700BF00ED00E0034B1A68B4
:103320001AB9034AD2F8D0241A60704768540020B2
:103330000040025808B5FFF7F1FF024B1868C0F3D0
:10334000806008BD68540020EFF3098305496833A5
:103350004A6B22F001024A6383F30988002383F356
:103360001188704700EF00E0302080F3118862B6CA
:103370000D4B0E4AD96821F4E0610904090C0A4397
:103380000B49DA60D3F8FC2042F08072C3F8FC20CD
:10339000084AC2F8B01F116841F0010111602022F3
:1033A000DA7783F82200704700ED00E00003FA05A9
:1033B00055CEACC5001000E0302310B583F3118862
:1033C0000E4B5B6813F4006314D0F1EE103AEFF388
:1033D00009844FF08073683CE361094BDB6B236623
:1033E00084F30988FFF7A0F910B1064BA36110BD63
:1033F000054BFBE783F31188F9E700BF00ED00E020
:1034000000EF00E02F0400083204000870B5BFF39D
:103410004F8FBFF36F8F1A4A0021C2F85012BFF3CB
:103420004F8FBFF36F8F536943F400335361BFF382
:103430004F8FBFF36F8FC2F88410BFF34F8FD2F856
:10344000803043F6E074C3F3C900C3F34E335B012D
:1034500003EA0406014646EA81750139C2F8605262
:10346000F9D2203B13F1200FF2D1BFF34F8F5369F4
:1034700043F480335361BFF34F8FBFF36F8F70BD41
:1034800000ED00E0FEE70000214B2248224A70B523
:10349000904237D3214BC11EDA1C121A22F00302CC
:1034A0008B4238BF00220021FDF7B6FD1C4A0023E5
:1034B000C2F88430BFF34F8FD2F8803043F6E07407
:1034C000C3F3C900C3F34E335B0103EA04060146AC
:1034D00046EA81750139C2F86C52F9D2203B13F1EA
:1034E000200FF2D1BFF34F8FBFF36F8FBFF34F8F1A
:1034F000BFF36F8F0023C2F85032BFF34F8FBFF37B
:103500006F8F70BD53F8041B40F8041BC0E700BF69
:10351000A45E0008B4580020B4580020B45800201D
:1035200000ED00E0074BD3F8D81021EA0001C3F802
:10353000D810D3F8002122EA0002C3F80021D3F802
:10354000003170470044025870B5D0E9244300228E
:103550004FF0FF359E6804EB42135101D3F8000988
:10356000002805DAD3F8000940F08040C3F80009CC
:10357000D3F8000B002805DAD3F8000B40F08040A8
:10358000C3F8000B013263189642C3F80859C3F818
:10359000085BE0D24FF00113C4F81C3870BD000086
:1035A000890141F02001016103699B06FCD41220CE
:1035B000FFF7F6B810B50A4C2046FEF795FD094B0B
:1035C000C4F89030084BC4F89430084C2046FEF7FD
:1035D0008BFD074BC4F89030064BC4F8943010BDF7
:1035E0006C54002000000840B85C0008085500201A
:1035F00000000440C45C000870B503780546012B48
:103600005CD1434BD0F89040984258D1414B0E21A9
:103610006520D3F8D82042F00062C3F8D820D3F850
:10362000002142F00062C3F80021D3F80021D3F852
:10363000802042F00062C3F88020D3F8802022F07E
:103640000062C3F88020D3F88030FEF7B3F9324B24
:10365000E360324BC4F800380023D5F89060C4F81A
:10366000003EC02323604FF40413A3633369002B8F
:10367000FCDA01230C203361FFF792F83369DB0792
:10368000FCD41220FFF78CF83369002BFCDA0026FB
:103690002846A660FFF758FF6B68C4F81068DB681F
:1036A000C4F81468C4F81C6883BB1D4BA3614FF0B9
:1036B000FF336361A36843F00103A36070BD194B3E
:1036C0009842C9D1134B4FF08060D3F8D82042F014
:1036D0000072C3F8D820D3F8002142F00072C3F87A
:1036E0000021D3F80021D3F8802042F00072C3F803
:1036F0008020D3F8802022F00072C3F88020D3F815
:103700008030FFF70FFF0E214D209EE7064BCDE7DF
:103710006C54002000440258401400400300200272
:10372000003C30C008550020083C30C0F8B5D0F847
:103730009040054600214FF000662046FFF730FF1D
:10374000D5F8941000234FF001128F684FF0FF302E
:10375000C4F83438C4F81C2804EB431201339F42E8
:10376000C2F80069C2F8006BC2F80809C2F8080B79
:10377000F2D20B68D5F89020C5F898306362102318
:103780001361166916F01006FBD11220FFF708F836
:10379000D4F8003823F4FE63C4F80038A36943F476
:1037A000402343F01003A3610923C4F81038C4F880
:1037B00014380B4BEB604FF0C043C4F8103B094B7F
:1037C000C4F8003BC4F81069C4F80039D5F8983043
:1037D00003F1100243F48013C5F89820A362F8BDEA
:1037E000945C000840800010D0F8902090F88A1077
:1037F000D2F8003823F4FE6343EA0113C2F800381C
:10380000704700002DE9F84300EB8103D0F8905099
:103810000C468046DA680FFA81F94801166806F00E
:103820000306731E022B05EB41134FF0000194BFFA
:10383000B604384EC3F8101B4FF0010104F1100319
:1038400098BF06F1805601FA03F3916998BF06F517
:10385000004600293AD0578A04F1580137434901FC
:103860006F50D5F81C180B430021C5F81C382B18D5
:103870000127C3F81019A7405369611E9BB3138A2F
:10388000928B9B08012A88BF5343D8F89820981838
:1038900042EA034301F140022146C8F89800284655
:1038A00005EB82025360FFF77BFE08EB8900C368DB
:1038B0001B8A43EA845348341E4364012E51D5F8D1
:1038C0001C381F43C5F81C78BDE8F88305EB491781
:1038D000D7F8001B21F40041C7F8001BD5F81C18CD
:1038E00021EA0303C0E704F13F030B4A28462146BF
:1038F00005EB83035A60FFF753FE05EB4910D0F840
:10390000003923F40043C0F80039D5F81C3823EA05
:103910000707D7E70080001000040002D0F89420C9
:103920001268C0F89820FFF70FBE00005831D0F899
:10393000903049015B5813F4004004D013F4001F89
:103940000CBF0220012070474831D0F89030490167
:103950005B5813F4004004D013F4001F0CBF022086
:103960000120704700EB8101CB68196A0B68136076
:103970004B6853607047000000EB810330B5DD6891
:10398000AA691368D36019B9402B84BF4023136020
:103990006B8A1468D0F890201C4402EB4110013C63
:1039A00009B2B4FBF3F46343033323F0030343EAA4
:1039B000C44343F0C043C0F8103B2B6803F003033B
:1039C000012B0ED1D2F8083802EB411013F4807F9E
:1039D000D0F8003B14BF43F0805343F00053C0F8CD
:1039E000003B02EB4112D2F8003B43F00443C2F823
:1039F000003B30BD2DE9F041D0F8906005460C4603
:103A000006EB4113D3F8087B3A07C3F8087B08D5C7
:103A1000D6F814381B0704D500EB8103DB685B681C
:103A20009847FA071FD5D6F81438DB071BD505EBE6
:103A30008403D968CCB98B69488A5A68B2FBF0F61E
:103A400000FB16228AB91868DA6890420DD2121A61
:103A5000C3E90024302383F3118821462846FFF769
:103A60008BFF84F31188BDE8F081012303FA04F28F
:103A70006B8923EA02036B81CB68002BF3D02146CC
:103A80002846BDE8F041184700EB81034A0170B5B4
:103A9000DD68D0F890306C692668E66056BB1A4441
:103AA0004FF40020C2F810092A6802F00302012A2C
:103AB0000AB20ED1D3F8080803EB421410F4807F49
:103AC000D4F8000914BF40F0805040F00050C4F812
:103AD000000903EB4212D2F8000940F00440C2F89A
:103AE00000090122D3F8340802FA01F10143C3F8B6
:103AF000341870BD19B9402E84BF40202060206862
:103B00001A442E8A8419013CB4FBF6F440EAC440FE
:103B100040F00050C6E700002DE9F843D0F890606F
:103B200005460C464F0106EB4113D3F8088918F0FF
:103B3000010FC3F808891CD0D6F81038DB0718D558
:103B400000EB8103D3F80CC0DCF81430D3F800E0AC
:103B5000DA68964530D2A2EB0E024FF000091A60E7
:103B6000C3F80490302383F31188FFF78DFF89F3A6
:103B7000118818F0800F1DD0D6F834380126A640E1
:103B8000334217D005EB84030134D5F89050D3F8B5
:103B90000CC0E4B22F44DCF8142005EB0434D2F856
:103BA00000E05168714514D3D5F8343823EA06068D
:103BB000C5F83468BDE8F883012303FA01F20389EC
:103BC00023EA02030381DCF80830002BD1D09847A8
:103BD000CFE7AEEB0103BCF81000834228BF0346D9
:103BE000D7F8180980B2B3EB800FE3D89068A0F142
:103BF000040959F8048FC4F80080A0EB0908984420
:103C0000B8F1040FF5D818440B4490605360C8E72E
:103C10002DE9F84FD0F8905004466E69AB691E400C
:103C200016F480586E6103D0BDE8F84FFEF7CCBAA9
:103C3000002E12DAD5F8003E9B0705D0D5F8003EDD
:103C400023F00303C5F8003ED5F80438204623F0DE
:103C50000103C5F80438FEF7E5FA370505D5204617
:103C6000FFF772FC2046FEF7CBFAB0040CD5D5F86E
:103C7000083813F0060FEB6823F470530CBF43F4BD
:103C8000105343F4A053EB6031071BD56368DB6826
:103C90001BB9AB6923F00803AB612378052B0CD16A
:103CA000D5F8003E9A0705D0D5F8003E23F003036F
:103CB000C5F8003E2046FEF7B5FA6368DB680BB135
:103CC00020469847F30200F1BA80B70226D5D4F80F
:103CD000909000274FF0010A09EB4712D2F8003B01
:103CE00003F44023B3F5802F11D1D2F8003B002B11
:103CF0000DDA62890AFA07F322EA0303638104EB0F
:103D00008703DB68DB6813B13946204698470137E3
:103D1000D4F89430FFB29B689F42DDD9F00619D5E4
:103D2000D4F89000026AC2F30A1702F00F0302F4FB
:103D3000F012B2F5802F00F0CA80B2F5402F09D101
:103D400004EB8303002200F58050DB681B6A974276
:103D500040F0B0803003D5F8185835D5E90303D5C5
:103D600000212046FFF746FEAA0303D50121204685
:103D7000FFF740FE6B0303D502212046FFF73AFE12
:103D80002F0303D503212046FFF734FEE80203D5B5
:103D900004212046FFF72EFEA90203D50521204667
:103DA000FFF728FE6A0203D506212046FFF722FE10
:103DB0002B0203D507212046FFF71CFEEF0103D598
:103DC00008212046FFF716FE700340F1A780E9079F
:103DD00003D500212046FFF79FFEAA0703D5012146
:103DE0002046FFF799FE6B0703D502212046FFF717
:103DF00093FE2F0703D503212046FFF78DFEEE0625
:103E000003D504212046FFF787FEA80603D5052128
:103E10002046FFF781FE690603D506212046FFF7FD
:103E20007BFE2A0603D507212046FFF775FEEB052A
:103E300074D520460821BDE8F84FFFF76DBED4F8D1
:103E400090904FF0000B4FF0010AD4F894305FFAD5
:103E50008BF79B689F423FF638AF09EB4713D3F8C7
:103E6000002902F44022B2F5802F20D1D3F8002996
:103E7000002A1CDAD3F8002942F09042C3F8002946
:103E8000D3F80029002AFBDB3946D4F89000FFF76D
:103E900087FB22890AFA07F322EA0303238104EB52
:103EA0008703DB689B6813B13946204698470BF1BE
:103EB000010BCAE7910701D1D0F80080072A02F16F
:103EC00001029CBF03F8018B4FEA18283FE704EB7F
:103ED000830300F58050DA68D2F818C0DCF80820B7
:103EE000DCE9001CA1EB0C0C00218F4208D1DB683F
:103EF0009B699A683A449A605A683A445A6029E73A
:103F000011F0030F01D1D0F800808C4501F10101BF
:103F100084BF02F8018B4FEA1828E6E7BDE8F88F66
:103F200008B50348FFF774FEBDE80840FFF744BA40
:103F30006C54002008B50348FFF76AFEBDE808404E
:103F4000FFF73ABA08550020D0F8903003EB411142
:103F5000D1F8003B43F40013C1F8003B7047000068
:103F6000D0F8903003EB4111D1F8003943F400133D
:103F7000C1F8003970470000D0F8903003EB4111D0
:103F8000D1F8003B23F40013C1F8003B7047000058
:103F9000D0F8903003EB4111D1F8003923F400132D
:103FA000C1F800397047000030B50433039C01723A
:103FB000002104FB0325C160C0E90653049B036391
:103FC000059BC0E90000C0E90422C0E90842C0E93D
:103FD0000A11436330BD00000022416AC260C0E99B
:103FE0000411C0E90A226FF00101FEF761BC000074
:103FF000D0E90432934201D1C2680AB9181D704752
:1040000000207047036919600021C2680132C26054
:10401000C269134482699342036124BF436A036106
:10402000FEF73ABC38B504460D46E3683BB1626919
:104030000020131D1268A3621344E36207E0237A91
:1040400033B929462046FEF717FC0028EDDA38BDC3
:104050006FF00100FBE70000C368C269013BC36069
:104060004369134482699342436124BF436A4361B5
:1040700000238362036B03B11847704770B5302388
:10408000044683F31188866A3EB9FFF7CBFF0546E5
:1040900018B186F31188284670BDA36AE26A13F846
:1040A000015B9342A36202D32046FFF7D5FF0023B2
:1040B00083F31188EFE700002DE9F84F04460E4620
:1040C000174698464FF0300989F311880025AA4613
:1040D000D4F828B0BBF1000F09D141462046FFF7C4
:1040E000A1FF20B18BF311882846BDE8F88FD4E9F1
:1040F0000A12A7EB050B521A934528BF9346BBF152
:10410000400F1BD9334601F1400251F8040B914294
:1041100043F8040BF9D1A36A403640354033A3621B
:10412000D4E90A239A4202D32046FFF795FF8AF387
:104130001188BD42D8D289F31188C9E730465A4662
:10414000FCF744FFA36A5E445D445B44A362E7E777
:1041500010B5029C0433017203FB0421C460C0E962
:1041600006130023C0E90A33039B0363049BC0E9E1
:104170000000C0E90422C0E90842436310BD00000A
:10418000026A6FF00101C260426AC0E904220022A3
:10419000C0E90A22FEF78CBBD0E904239A4201D180
:1041A000C26822B9184650F8043B0B6070470023E0
:1041B0001846FAE7C3680021C2690133C360436946
:1041C000134482699342436124BF436A4361FEF70B
:1041D00063BB000038B504460D46E3683BB1236974
:1041E00000201A1DA262E2691344E36207E0237A09
:1041F00033B929462046FEF73FFB0028EDDA38BDEB
:104200006FF00100FBE7000003691960C268013A22
:10421000C260C269134482699342036124BF436A46
:10422000036100238362036B03B1184770470000EA
:1042300070B530230D460446114683F31188866A13
:104240002EB9FFF7C7FF10B186F3118870BDA36ABE
:104250001D70A36AE26A01339342A36204D3E16949
:1042600020460439FFF7D0FF002080F31188EDE7E6
:104270002DE9F84F04460D46904699464FF0300A16
:104280008AF311880026B346A76A4FB949462046EB
:10429000FFF7A0FF20B187F311883046BDE8F88F03
:1042A000D4E90A073A1AA8EB0607974228BF17462F
:1042B000402F1BD905F1400355F8042B9D4240F8CF
:1042C000042BF9D1A36A40364033A362D4E90A2310
:1042D0009A4204D3E16920460439FFF795FF8BF336
:1042E00011884645D9D28AF31188CDE729463A4646
:1042F000FCF76CFEA36A3D443E443B44A362E5E701
:10430000D0E904239A4217D1C3689BB1836A8BB169
:10431000043B9B1A0ED01360C368013BC360C369A2
:104320001A4483699A42026124BF436A03610023ED
:1043300083620123184670470023FBE700F064BA4C
:10434000014B586A704700BF000C0040034B00222D
:1043500058631A610222DA60704700BF000C004007
:10436000014B0022DA607047000C0040014B58639B
:10437000704700BF000C0040024B034A1A60034A1A
:104380005A607047BC550020B85800200000022039
:10439000074B494210B55C68201A08401968821A18
:1043A0008A4203D3A24201D85A6010BD0020FCE724
:1043B000BC55002008B5302383F31188FFF7E8FFD0
:1043C000002383F3118808BD04480121044B0360D6
:1043D0000023C0E901330C3000F016B9C4550020A9
:1043E000B5430008CB1D083A23F00703591A521AA7
:1043F000012110B4D2080024C0E9004384600C30CD
:104400001C605A605DF8044B00F0FEB82DE9F84FCF
:10441000364ECD1D0F46002818BF0646082A4FEA23
:10442000D50538BF082206F10C08341D91464046D8
:1044300000F006F909F10701C9F1000E22462468CF
:104440006CB9404600F006F93368CBB30822494600
:10445000E8009847044698B340E9026730E004EB6F
:10446000010CD4F804A00CEA0E0C0AF10100ACF126
:10447000080304EBC0009842E0D9A0EB0C0CB5EBAC
:10448000EC0F4FEAEC0BD9D89C421CD204F1080285
:10449000AB45A3EB02024FEAE202626009D9691C54
:1044A000ED43206803EBC1025D44556043F83100E1
:1044B00022601C465F60404644F8086B00F0CAF872
:1044C0002046BDE8F88FAA45216802D11160234635
:1044D000EFE7013504EBC50344F8351003F108019B
:1044E000401AC01058601360F1E700BFC4550020A7
:1044F000F8B550F8043C044650F8085CA0F10806F2
:1045000007332F1D0C35DB0840F8043C284600F02B
:1045100097F83B469F421A6801D0B34228D20AB1AD
:10452000964225D244F8082C54F8042C1E6001321F
:1045300054F8081C06EBC200814206D148680244C8
:1045400044F8042C0A6844F8082C5868411C03EB12
:10455000C1018E4207D154F8042C013202445A6042
:1045600054F8082C1A602846BDE8F84000F072B8EC
:104570001346CFE7FEE7000070B51B4B002504464D
:1045800086B058600E4685620163FEF7EDFE04F1C9
:104590001003A560E562C4E904334FF0FF33C4E9BA
:1045A0000044C4E90635FFF7CBFE2B46024604F172
:1045B00034012046C4E9082380230C4A2565FEF710
:1045C000F9F801230A4AE0600092037568467268B0
:1045D0000192B268CDE90223064BCDE90435FEF71E
:1045E00011F906B070BD00BF80380020D05C000813
:1045F000D55C000875450008024AD36A1843D062AA
:10460000704700BF18360020C0E900008160704785
:104610008368013B002B10B583600CDA074BDC6824
:104620004368A061206063601C6044600520FEF761
:1046300033F8A06910BD0020FCE700BF1836002049
:1046400008B5302383F31188FFF7E2FF002383F3DB
:10465000118808BD08B5302383F3118883680133BE
:10466000002B836007DC036800211A680260506039
:104670001846FEF73DF8002383F3118808BD0000BB
:104680004B6843608B688360CB68C3600B69436190
:104690004B6903628B6943620B68036070470000DB
:1046A00008B53C4B40F2FF713B48D3F888200A43E1
:1046B000C3F88820D3F8882022F4FF6222F0070292
:1046C000C3F88820D3F88820D3F8E0200A43C3F841
:1046D000E020D3F808210A43C3F808212F4AD3F871
:1046E00008311146FFF7CCFF00F5806002F11C0194
:1046F000FFF7C6FF00F5806002F13801FFF7C0FF49
:1047000000F5806002F15401FFF7BAFF00F5806008
:1047100002F17001FFF7B4FF00F5806002F18C0137
:10472000FFF7AEFF00F5806002F1A801FFF7A8FFD8
:1047300000F5806002F1C401FFF7A2FF00F5806080
:1047400002F1E001FFF79CFF00F5806002F1FC013F
:10475000FFF796FF02F58C7100F58060FFF790FF80
:1047600000F01EF90E4BD3F8902242F00102C3F87C
:104770009022D3F8942242F00102C3F89422052239
:10478000C3F898204FF06052C3F89C20054AC3F844
:10479000A02008BD0044025800000258DC5C00085C
:1047A00000ED00E01F00080308B500F013FBFDF763
:1047B000DBFF104BD3F8DC2042F04002C3F8DC20D2
:1047C000D3F8042122F04002C3F80421D3F80431C5
:1047D000094B1A6842F008021A601A6842F0040293
:1047E0001A60FEF79BFDFEF7D1FCBDE80840FEF71E
:1047F0004BBA00BF0044025800180248012070471D
:104800000020704770470000114BD3F8E82042F0B9
:104810000802C3F8E820D3F8102142F00802C3F8D8
:1048200010210C4AD3F81031D36B43F00803D36343
:10483000C722094B9A624FF0FF32DA6200229A6176
:104840005A63DA605A6001225A611A60704700BFE9
:10485000004402580010005C000C0040094A08B5F2
:104860001169D3680B40D9B29B076FEA010111614E
:1048700007D5302383F31188FDF790FF002383F3DE
:10488000118808BD000C0040064BD3F8DC20024321
:10489000C3F8DC20D3F804211043C3F80401D3F893
:1048A000043170470044025808B53C4B4FF0FF31CB
:1048B000D3F8802062F00042C3F88020D3F8802033
:1048C00002F00042C3F88020D3F88020D3F884207F
:1048D000C3F88410D3F884200022C3F88420D3F8CE
:1048E0008400D86F40F0FF4040F4FF0040F4DF4008
:1048F00040F07F00D867D86F20F0FF4020F4FF0021
:1049000020F4DF4020F07F00D867D86FD3F888000C
:104910006FEA40506FEA5050C3F88800D3F888001F
:10492000C0F30A00C3F88800D3F88800D3F89000D9
:10493000C3F89010D3F89000C3F89020D3F89000FB
:10494000D3F89400C3F89410D3F89400C3F89420DB
:10495000D3F89400D3F89800C3F89810D3F89800CF
:10496000C3F89820D3F89800D3F88C00C3F88C10C3
:10497000D3F88C00C3F88C20D3F88C00D3F89C00BB
:10498000C3F89C10D3F89C10C3F89C20D3F89C303B
:10499000FCF778FDBDE8084000F0E0B9004402589B
:1049A00008B50122534BC3F80821534BD3F8F42028
:1049B00042F00202C3F8F420D3F81C2142F00202B4
:1049C000C3F81C210222D3F81C314C4BDA605A6820
:1049D0009104FCD54A4A1A6001229A60494ADA6079
:1049E00000221A614FF440429A61444B9A69920442
:1049F000FCD51A6842F480721A603F4B1A6F12F4A9
:104A0000407F04D04FF480321A6700221A671A6878
:104A100042F001021A60384B1A685007FCD5002298
:104A20001A611A6912F03802FBD1012119604FF0A6
:104A3000804159605A67344ADA62344A1A611A6806
:104A400042F480321A602C4B1A689103FCD51A6824
:104A500042F480521A601A689204FCD52C4A2D49FF
:104A60009A6200225A63196301F57C01DA6301F24C
:104A7000E71199635A64284A1A64284ADA621A6864
:104A800042F0A8521A601C4B1A6802F02852B2F188
:104A9000285FF9D148229A614FF48862DA61402296
:104AA0001A621F4ADA641F4A1A651F4A5A651F4A6A
:104AB0009A6532231E4A1360136803F00F03022B1A
:104AC000FAD10D4A136943F003031361136903F02C
:104AD0003803182BFAD14FF00050FFF7D5FE4FF0F6
:104AE0008040FFF7D1FE4FF00040BDE80840FFF7DF
:104AF000CBBE00BF0080005100440258004802585D
:104B000000C000F0020000010000FF0100889008D2
:104B10002220400063020901470E0508DD0BBF019A
:104B200020000020000001100910E0000001011029
:104B3000002000524FF0B04208B5D2F8883003F0A0
:104B40000103C2F8883023B1044A13680BB15068DE
:104B50009847BDE80840FEF72FBC00BFDC55002099
:104B60004FF0B04208B5D2F8883003F00203C2F823
:104B7000883023B1044A93680BB1D0689847BDE8E8
:104B80000840FEF719BC00BFDC5500204FF0B042D2
:104B900008B5D2F8883003F00403C2F8883023B196
:104BA000044A13690BB150699847BDE80840FEF705
:104BB00003BC00BFDC5500204FF0B04208B5D2F86E
:104BC000883003F00803C2F8883023B1044A93699F
:104BD0000BB1D0699847BDE80840FEF7EDBB00BFB8
:104BE000DC5500204FF0B04208B5D2F8883003F011
:104BF0001003C2F8883023B1044A136A0BB1506A1B
:104C00009847BDE80840FEF7D7BB00BFDC55002041
:104C10004FF0B04310B5D3F8884004F47872C3F86D
:104C20008820A30604D5124A936A0BB1D06A98472C
:104C3000600604D50E4A136B0BB1506B98472106E2
:104C400004D50B4A936B0BB1D06B9847E20504D5A2
:104C5000074A136C0BB1506C9847A30504D5044A5E
:104C6000936C0BB1D06C9847BDE81040FEF7A4BB25
:104C7000DC5500204FF0B04310B5D3F8884004F461
:104C80007C42C3F88820620504D5164A136D0BB127
:104C9000506D9847230504D5124A936D0BB1D06D22
:104CA0009847E00404D50F4A136E0BB1506E984735
:104CB000A10404D50B4A936E0BB1D06E98476204E1
:104CC00004D5084A136F0BB1506F9847230404D5DD
:104CD000044A936F0BB1D06F9847BDE81040FEF7C0
:104CE0006BBB00BFDC55002008B5034800F038FD61
:104CF000BDE80840FEF760BB5C56002008B50348DD
:104D0000FCF7D2FDBDE80840FEF756BB6424002046
:104D100008B50348FCF7C8FDBDE80840FEF74CBBEA
:104D2000D024002008B50348FCF7BEFDBDE80840CC
:104D3000FEF742BB3C25002008B50348FCF7B4FD54
:104D4000BDE80840FEF738BBA825002008B5FFF7EE
:104D500085FDBDE80840FEF72FBB0000062108B521
:104D60000846FCF727FE06210720FCF723FE062154
:104D70000820FCF71FFE06210920FCF71BFE062178
:104D80000A20FCF717FE06211720FCF713FE062168
:104D90002820FCF70FFE09217A20FCF70BFE0921E1
:104DA0007C20FCF707FE07213220FCF703FE0C21D4
:104DB0002520FCF7FFFD0C212720FCF7FBFD0C2133
:104DC0003520FCF7F7FD0C215220BDE80840FCF728
:104DD000F1BD000008B5FFF767FD00F015FAFCF71C
:104DE000A7FF00F003FAFDF77DF9FDF74FF8FFF795
:104DF00009FDBDE80840FFF7A1BA00000379052BC3
:104E000005BF836A002001204B6004BF4FF400738C
:104E10000B60704770B55D1E866A04460D44B5424E
:104E200005D9436B43F080034363012070BD062521
:104E3000057100F047FC05232371F7E770B55D1E8F
:104E4000866A04460D44B54205D9436B43F080039E
:104E50004363012070BD0725057100F059FC05234F
:104E60002371F7E738B505790446052D05D10823E8
:104E7000037100F073FC257138BD0120FCE70000D0
:104E80000323F0B5037185B0044600F00DFA00224B
:104E90002046114600F052FA4FF4D57203AB0821B8
:104EA000204600F06DFA0246B8B901232363039B44
:104EB000C3F30323012B09D103AB3721204600F0B4
:104EC0005FFA18B9A44B039A1340ABB120460125F1
:104ED00000F01CFA0223237137E103AB00223721D3
:104EE000204600F04DFA28B99B4A039B1A40002A3D
:104EF00000F0A78002232363236B03F00F03022B30
:104F000040F0A9806425954E42F21070FDF790FCA8
:104F100003AB32460121204600F01CFA0028D5D10F
:104F2000039B002B80F293805A0003D5236B43F040
:104F300010032363002204F108030221204600F03D
:104F40007DFA02460028C1D104F13803032120462E
:104F500000F016FA0028B9D104F11805A26B092156
:104F600020462B4600F06AFA0028AFD102ABA26BB4
:104F70000721204600F004FA06460028A6D1236B3C
:104F800003F00F03022B40F08F807E227F21284602
:104F900000F0F4FB012840F28780E76B42F21070CA
:104FA000FDF746FC08234FF4007239462046009670
:104FB00000F060FA002889D1384600F02DFC236B00
:104FC000A06203F00F03022B72D103AB644A0621E7
:104FD000204600F0D5F9002871D15F49039B1940A4
:104FE000B1FA81F14909204600F070F902AB4FF4A3
:104FF00000721021204600F0C3F9054600287FF416
:1050000065AF554E029B33427FF460AF236B13F0C4
:105010000E0F03F00F0273D0022A7FF457AFE36A3A
:105020001978012900F09480022900F0938000296A
:1050300000F089804B4F204600F06EF903AB3A46F2
:1050400076E011462046226300F078F954E7013DEE
:105050007FF45AAF3AE7444D6426444A3E4F012B51
:1050600018BF154603AB00223721204600F088F90F
:1050700000287FF42BAF039B3B427FF427AF03ABA9
:105080002A462921204600F065F900287FF41EAF4A
:10509000039B002BFFF648AF013E3FF417AF42F2EF
:1050A0001070FDF7C5FBDDE7284600F089FB86E7B9
:1050B0007E227F212846E66B00F060FB08B90021C4
:1050C00091E700234022314620460093062300F05A
:1050D000D1F90028F3D1B3895BBA9B07EFD5244BF4
:1050E0004022314620460093062300F0C3F90028F1
:1050F000E5D1317C01F00F010F3918BF012172E7B2
:10510000E36A1978F9B101297FF4E0AE204600F096
:1051100003F903ABA26B3721204600F031F90028D8
:105120007FF4D4AE039B33427FF4D0AE03AB0222B4
:105130000621204600F024F900287FF4C7AE039B27
:1051400033427FF4C3AE05232371284605B0F0BD7A
:10515000084F70E7084F6EE708E0FFFD0080FFC0D2
:105160000001B9030000B7030080FF500000108069
:10517000F1FFFF800001B7030002B70337B5044613
:105180000C4D01ABA26B0D21204600F0F9F878B967
:10519000019B2B420BD1C3F34323042B08D0053BC7
:1051A000022B04D84FF47A70FDF742FBE9E70120A7
:1051B00003B030BD08E0FFFD70B53023054683F332
:1051C000118803790024022B03D184F3118820462F
:1051D00070BD0423037184F311880226FFF7CEFF0C
:1051E0000446284600F092F82E71F0E700F042B82D
:1051F000044B03600123037100234363C0E90A33B6
:10520000704700BF105E00080023054A19460133AD
:10521000102BC2E9001102F10802F8D1704700BF5B
:10522000DC550020836CC26A8B42506810B506D9E9
:105230005A1E4C0002EB4103B3FBF4F3184410BDBB
:1052400001F001038A0748BF43F002034A0748BF41
:1052500043F008030A0748BF43F00403CA0648BFE7
:1052600043F010038A06426B48BF43F02003134308
:105270004363704710B5074C2046FFF7B9FF064B54
:105280000022C4E91023054BA364054BE363054BDF
:10529000E36410BD5C5600200024024800B4C4043E
:1052A000B0560020B058002010B5446C0649FFF7F6
:1052B000B9FF6060236842F2107043F0030323607B
:1052C000BDE81040FDF7B4BA801A06000129F8B510
:1052D000466C0B4F09D175680A493D40FFF7A2FFA4
:1052E000054345F480557560F8BD746806493C4037
:1052F000FFF798FF044344F480547460F4E700BF60
:1053000000ECFFFF80F0FA0240787D01436C002240
:105310005A601A6070470000426C0129536823F4F8
:10532000404304D0022905D001B95360704743F4CB
:105330008043FAE743F40043F7E70000436C41F48D
:1053400080519A60D9605A6B1206FCD580229A630C
:105350007047000010B541F48851446CA260E160D0
:10536000616B11F04502FBD0A26311F0040203D07F
:10537000FFF766FF012010BD616910461960FAE76A
:1053800010B541F48851446CA260E160616B11F08A
:105390004502FBD0A26311F0050203D0FFF750FFD6
:1053A000012010BD616910461960FAE773B5134614
:1053B00004460E46302282F31188426CD26B32B121
:1053C0004FF0FF3140300193FDF73EFA019B606CD6
:1053D00000220265C263C262456B15F4807504D178
:1053E00085F31188012002B070BD4FF0FF31816359
:1053F00082F31188012E06D90C21204602B0BDE8A7
:105400007040FFF7BDBF1046EDE7000073B5446C78
:105410000E4600250192616BA1632565E562FFF7E9
:105420000FFF012E07D9019B2A460C2102B0BDE8CF
:105430007040FFF7A5BF02B070BD000010B541F489
:105440009851446CA260E160616B11F04502FBD0A1
:10545000A26311F03F0203D0FFF7F2FE012010BD5E
:10546000216A10461960E1695960A1699960616912
:10547000D960F4E72DE9F74304460191006D01A9D5
:105480001746984600F0D8F9064600284AD0626CC4
:105490002046DDF804905568C5F3090501356B0019
:1054A000A56CB5FBF3F54FF47A73B5FBF3F55D43EB
:1054B0005562FFF763FE50BB636C4FF0FF3201256E
:1054C0004146C3F8589020461D659A634FF4957283
:1054D000DA6342F207029F62DA62E36C0A9AFFF72C
:1054E0004FFFA0B9E26C104B11680B407BB9294605
:1054F0002046FFF75BFF054648B92E463A4601991C
:10550000206D00F0D1F9304603B0BDE8F0833A4693
:105510000199206D00F0C8F9E26C01212046FFF7E7
:1055200075FFF0E70126EEE708E0FFFD2DE9F74300
:105530001F46436C01924FF47A725D6804468846B8
:10554000C5F3090501356E00856CB5FBF6F5B5FBB5
:10555000F2F555435D62FFF711FE20B101252846A3
:1055600003B0BDE8F0837E0201A9206D324600F051
:1055700063F905460028F1D0636C019AD4F84C9089
:105580009A6501221A654FF0FF329A634FF49572C3
:10559000DA639E62236BDB064B4658BF4FEA48280E
:1055A000012F42461BD912212046FFF7E9FEC0B960
:1055B000D9F80020104B13409BB9636C42F2930260
:1055C00039462046DA62E26CFFF7F0FE804640B9C9
:1055D00032460199206D454600F066F9BFE711217A
:1055E000E2E732460199206D00F05EF9E26C39463F
:1055F0002046FFF70BFFB2E708E0FFFD2DE9F3417E
:105600001F46436C01924FF47A725D6804468846E7
:10561000C5F3090501356E00856CB5FBF6F5B5FBE4
:10562000F2F555435D62FFF7A9FD20B1012528463B
:1056300002B0BDE8F0817E0201A9206D324600F083
:1056400041F905460028F1D0636C019A9A65012260
:105650001A654FF0FF329A634FF48D72DA639E62DF
:10566000236BE66CDB06334658BF4FEA4828012F10
:10567000424619D919212046FFF782FEB0B9326897
:105680000F4B134093B9636C42F2910239462046A6
:10569000DA62E26CFFF78AFE064638B901993546B0
:1056A000206D00F04BF9C2E71821E4E70199206D65
:1056B00000F044F9E26C39462046FFF7A7FEB6E752
:1056C00008E0FFFD12F0030F2DE9F04107460C46FC
:1056D00015461E4617D00E44B44202D10020BDE844
:1056E000F0810123FA6B21463846FFF71FFF00289F
:1056F000F5D128464FF40072F96B05F500750134B9
:10570000FBF764FCE8E7BDE8F041FFF70FBF0000DE
:1057100012F0030F2DE9F04107460C4615461E46D0
:1057200017D00E44B44202D10020BDE8F0812946D2
:105730004FF40072F86B05F50075FBF747FC012389
:10574000FA6B21463846FFF759FF0028EDD10134A6
:10575000E8E7BDE8F041FFF751BF000000207047C7
:10576000302310B583F311880024436C4030214668
:10577000DC63FDF777F884F3118810BD01F01F0397
:10578000F0B502F01F0456095A1C0123B6EB511F55
:1057900050F8265003FA02F34FEA511703F1FF3392
:1057A0003DBF50F82720C4F12000134003EA050054
:1057B0003BBF03FA00F225FA04F0E0401043F0BDCD
:1057C00070B57E227F210546FFF7D8FF18B101286A
:1057D00019D0002070BD3E2249212846FFF7CEFF98
:1057E0002F22044631212846FFF7C8FF0646013420
:1057F0005022023653212846B440FFF7BFFF093834
:1058000004FA00F0E6E7302245212846FFF7B6FF0C
:1058100001308002DEE7000090F8D63090F8D72003
:105820001B0403EB026390F8D42090F8D5001344D6
:1058300003EB002070470000F8B50F4615460446FC
:1058400048B905F11F010126386821F01F01FDF755
:1058500041FD3046F8BD427B29463868FDF7D0FC53
:1058600006460028EDD13B686360A368AB4210D2C6
:1058700013B12068FDF7C0FC637B28462BB1FDF710
:10588000B7FC206020B9A060E3E7FDF77BFCF8E7F8
:10589000A560206805F11F01012621F01F01386075
:1058A000FDF718FD2673D4E710B5044640B1006833
:1058B000884205D1606808B1FBF788FB0023237399
:1058C00010BD0000F8B50F461446054648B904F16E
:1058D0001F010126386821F01F01FDF70DFD30463C
:1058E000F8BD427B21463868FDF78AFC0646002851
:1058F000EDD1AB68A34210D213B12868FDF77CFC50
:105900006B7B20462BB1FDF773FC286020B9A860A3
:10591000E5E7FDF737FCF8E7AC60396819B12246D6
:105920002868FBF753FB286804F11F01012621F0CA
:105930001F013860FDF7E0FC2E73D0E720B103684B
:105940008B4204BF002303737047000010B5013978
:105950000244904201D1002005E0037811F8014F84
:10596000A34201D0181B10BD0130F2E7034611F825
:10597000012B03F8012B002AF9D1704753544D3302
:105980003248373F3F3F0053544D33324837337826
:105990002F3732780053544D3332483734332F3752
:1059A00035332F373530000001105A0003105900ED
:1059B0000120580003205600100002400800024059
:1059C0000008024000000B002800024008000240CE
:1059D0000408024006010C0040000240080002409A
:1059E0000808024010020D00580002400800024062
:1059F0000C08024016030E00700002400C0002402A
:105A00001008024000040F00880002400C00024011
:105A10001408024006051000A00002400C000240DD
:105A20001808024010061100B80002400C000240A5
:105A30001C08024016072F00100402400804024010
:105A400020080240000838002804024008040240F0
:105A500024080240060939004004024008040240BC
:105A600028080240100A3A00580402400804024084
:105A70002C080240160B3B00700402400C0402404C
:105A800030080240000C3C00880402400C04024034
:105A900034080240060D4400A00402400C040240F9
:105AA00038080240100E4500B80402400C040240C1
:105AB0003C080240160F460000960000000000005F
:105AC00000000000000000000000000000000000D6
:105AD00000000000F11C0008DD1C0008191D000872
:105AE000051D0008111D0008FD1C0008E91C000828
:105AF000D51C0008251D000800000000091E000834
:105B0000F51D0008311E00081D1E0008291E000892
:105B1000151E0008011E0008ED1D00083D1E0008AE
:105B200000000000010000000000000063300000E1
:105B30002C5B0008703600208038002041726475AC
:105B400050696C6F740025424F415244252D424CE0
:105B5000002553455249414C250000000200000039
:105B600000000000292000089920000840004000A3
:105B700030510020405100200200000000000000D1
:105B80000300000000000000E12000080000000009
:105B90001000000050510020000000000100000033
:105BA000000000006C54002001010200252C0008B8
:105BB000352B0008D12B0008B52B0008430000004E
:105BC000C45B000809024300020100C0320904005E
:105BD000000102020100052400100105240100015A
:105BE000042402020524060001070582030800FFC1
:105BF00009040100020A000000070501024000003C
:105C0000070581024000000012000000105C00083F
:105C10001201100102000040091241570002010266
:105C2000030100000403090425424F4152442500AA
:105C300041524B5F5049365800303132333435369B
:105C400037383941424344454600000000000020F7
:105C5000000002000200000000000030000004000C
:105C600008000000000000240000080004000000FC
:105C70000004000000FC00000200000000000430EE
:105C80000080000008000000000000380000010053
:105C900001000000000000003D220008F52400087B
:105CA000A125000840004000A4550020A455002074
:105CB00001000000B45500208000000040010000F9
:105CC00008000000000100000010000008000000B3
:105CD0006D61696E0069646C650000000000802AD7
:105CE00000020000AAAAAAAA00000024FFFF0000E8
:105CF0000000000000A00A0000A200A000000000B8
:105D0000AAAAAAAA00510050FFFF000000000977CC
:105D1000000000990000090200000000AAAAAAAA37
:105D200000000601FFFF00000000000080000800E6
:105D300020A00A0000000000AAAAAAAA104005009C
:105D4000FFFF0000000800BB7700000040142200A5
:105D500028000000AAAAAAAA00001100FFFF000064
:105D60000000000007070000002001000000000004
:105D7000AAAAAAAA00100200FFFF00000000000764
:105D8000000000000000900000000000AAAAAAAADB
:105D900000004000FFFF00000000000000A0000025
:105DA0000004000000000000AAAAAAAA0004000043
:105DB000FFFF0000000000000000000000000400E1
:105DC00000000000AAAAAAAA00000400FFFF000029
:105DD00000000000000000000000000000000000C3
:105DE000AAAAAAAA00000000FFFF0000000000000D
:105DF000000000000000000000000000AAAAAAAAFB
:105E000000000000FFFF0000000000000000000094
:105E100000000000FD47000801480008814E00080E
:105E2000B9510008154E00083D4E0008654E0008A7
:105E3000FD4D0008000000003A00000000000000D6
:105E400000001A0000000000FF0000008838002059
:105E5000A82500203C250020D024002000000000C0
:105E60007C59000883040000875900085004000092
:105E700095590008009600000000080096000000F8
:105E80000008000004000000245C0008000000007E
:105E90000000000000000000000000000000000002
:045EA00000000000FE
:00000001FF
